:1000000012C02CC02BC02BC029C028C027C026C0BE
:1000100025C0FFC023C022C021C020C01FC01EC0F9
:100020001DC01CC01BC011241FBECFE5D4E0DEBF25
:10003000CDBF10E0A0E6B0E0E2EDF2E102C0059035
:100040000D92A038B107D9F712E0A0E8B0E001C0E6
:100050001D92A93DB107E1F792D039C9D1CF1F92C6
:100060000F920FB60F9211242F938F939F93EF93BC
:10007000FF93E091D702F091D802EA53FF4F8081BD
:1000800090E09BBD8ABD8091D7029091D8020196E5
:100090009093D8028093D7028091D7029091D80292
:1000A0008050924020F01092D8021092D702FF9117
:1000B000EF919F918F912F910F900FBE0F901F90F6
:1000C00018950F931F93DF93CF9300D0CDB7DEB772
:1000D0008C018CE990E09DD6C8014AD48093D60269
:1000E000882311F081E044C086EC90E060E072E08B
:1000F0008E010F5F1F4FA80145D38093D60288233E
:1001000011F083E035C080E889BF20E02223A9F404
:100110008091D7029091D8028F3F9105C9F3C0F327
:1001200086EC90E060E071E0A8012CD389819A818F
:100130008F3F9105B1F0A8F021E08091D702909116
:10014000D8028F3F910509F008F786EC91E060E056
:1001500071E0A80117D389819A818F3F910509F039
:10016000B8F619BE80E090E054D68093D60280E0C5
:100170000F900F90CF91DF911F910F91089583E021
:1001800081BB12BA18BA82E087BB81E88FBD89E0D3
:100190008EBD1DBC1CBC1BBC1ABC8BE085BD14BC39
:1001A00084E083BD83B7856083BF89B7816089BFE1
:1001B00012BE78941AD842D880938000813041F4DE
:1001C000909A80E690E07DDF89B7816089BF909842
:1001D00080918000823041F4919A88E690E071DF4E
:1001E00089B7816089BF919880918000833031F414
:1001F00080E790E066DF89B7816089BF80918000E9
:100200008430C9F688E790E05CDF89B7816089BFF8
:10021000D2CF1F920F920FB60F9211242F933F93BC
:100220004F935F936F937F938F939F93AF93BF93FE
:10023000EF93FF93E1D7FF91EF91BF91AF919F9122
:100240008F917F916F915F914F913F912F910F907F
:100250000FBE0F901F901895DF92EF92FF920F93B1
:100260001F93D82E7A018B0187FF0BC087E740E0F0
:1002700050E060E070E0F0DF823008F040C08FE7CF
:10028000D822C29A8FEF8FB9779BFECF8FB1C298D9
:100290008FEF8FB9779BFECF8FB1DFB8779BFECF03
:1002A000812F9927AA27BB278FB9779BFECFC8013B
:1002B000AA27BB278FB9779BFECFBB27A12F902FF3
:1002C0008F2D8FB9779BFECFEFB8779BFECF80E461
:1002D000D81611F485E906C088E4D81611F487E829
:1002E00001C081E08FB9779BFECF9AE02FEF2FB945
:1002F000779BFECF8FB187FF02C09150C1F71F914E
:100300000F91FF90EF90DF900895EF92FF920F937F
:100310001F93CF93DF937C01E9018091810083FDDE
:1003200007C039E0440F551F661F771F3A95D1F774
:1003300081E592DF882309F03AC080E49CE93FEF31
:100340003FB9779BFECF2FB12F3F19F40197C1F72B
:100350002EC02E3F61F5222733272C1B3D0B2E5F2D
:100360003D4F201B310B209739F08FEF8FB9779BD2
:10037000FECF9FB12197D1F7E114F10471F09FEF07
:100380009FB9779BFECF8FB1F7018083015010405A
:1003900021F00894E11CF11CF3CF8FEF8FB9779B0C
:1003A000FECF9FB121503040C9F790E001C091E0ED
:1003B000C29A8FEF8FB9779BFECF8FB1892FDF91D4
:1003C000CF911F910F91FF90EF900895AF92BF9240
:1003D000CF92DF92EF92FF920F931F93DF93CF9311
:1003E00000D000D0CDB7DEB7CCD6C29A8AE09FEF5E
:1003F0009FB9779BFECF2FB18150D1F780E440E0C9
:1004000050E060E070E028DF813009F074C088E4DB
:100410004AEA51E060E070E01FDF813009F045C03A
:100420006E010894C11CD11C76019FEF9E012B5FC9
:100430003F4F9FB9779BFECF8FB1F70181937F012B
:10044000E217F307B1F78B81813009F054C08C813A
:100450008A3A09F050C000E117E2A8ECAA2EB12CAC
:1004600007C0C5010197F1F70150104009F443C0DE
:1004700089EE40E050E060E070E4EEDE882389F72A
:1004800056C09FEF9FB9779BFECF8FB1F601819346
:100490006F01EE15FF05B1F7898186FD03C0F4E019
:1004A000FF2E2AC0ECE0FE2E27C089EE40E050E08F
:1004B00060E070E0D1DE823028F071E4E72EFF24A6
:1004C000F39404C069EEE62E52E0F52E00E117E247
:1004D00048ECC42ED12C06C0C6010197F1F701509B
:1004E000104049F08E2D40E050E060E070E0B4DE56
:1004F000882391F726C0FF24F0928100C29A8FEFE3
:100500008FB9779BFECF8FB180E0FF2009F481E0A7
:100510000F900F900F900F90CF91DF911F910F913F
:10052000FF90EF90DF90CF90BF90AF9008958AE753
:1005300040E050E060E070E08FDE882309F4A1CF56
:10054000DACF80E540E052E060E070E085DE8823AD
:1005500091F6D2CFCF92DF92EF92FF920F931F933B
:10056000CF93DF936C01C0918200D0918300FC0196
:1005700011821082248135814681578121303105D5
:100580004105510509F45AC08E819F81A885B9851E
:10059000281739074A075B0708F050C021153105B5
:1005A0004105510539F48881833021F42E853F853A
:1005B00048895989F6012087318742875387211559
:1005C00031054105510579F18EEFE82E8FEFF82EB8
:1005D0008FEF082F8FEF182FE20EF31E041F151F49
:1005E0008E819F81A885B9850297A109B109E81676
:1005F000F9060A071B0728F020E030E040E050E051
:1006000016C02A8130E040E050E0C801B7011ED694
:100610009B01AC018A899B89AC89BD89280F391F50
:100620004A1F5B1F04C02E853F8548895989F60102
:10063000248735874687578780E001C081E0DF91B6
:10064000CF911F910F91FF90EF90DF90CF90089581
:100650000F931F93DF93CF9300D000D0CDB7DEB7B9
:100660008B019C01E0918200F09183006230710562
:100670008105910508F477C086819781A085B185B1
:10068000081719072A073B0708F06DC080818230E0
:1006900021F0833009F067C022C07727632F522FE3
:1006A000412F82859385A485B585480F591F6A1F00
:1006B0007B1F98013070220F331FCE01019602E09C
:1006C00010E023DE882309F04EC09A8180E0298162
:1006D00030E0822B932B9C0140E050E048C0B901F0
:1006E000A801A7E07695679557954795AA95D1F704
:1006F00082859385A485B585480F591F6A1F7B1F86
:1007000098012F773070220F331F220F331FCE0135
:10071000019604E010E0F9DD882329F58C8190E052
:10072000A0E0B0E0582F4427332722278B8190E0A8
:10073000A0E0B0E0DC0199278827282B392B4A2B31
:100740005B2B898190E0A0E0B0E0282B392B4A2B6D
:100750005B2B9A8180E0A0E0B0E0282B392B4A2B5C
:100760005B2B5F7004C021E030E040E050E0B90155
:10077000CA010F900F900F900F90CF91DF911F91B2
:100780000F9108954F925F926F927F928F929F92F6
:10079000AF92BF92CF92DF92EF92FF920F931F938F
:1007A000CF93DF933C016B014A01C0918200D0914D
:1007B0008300FA0111821082209711F486E0C7C0ED
:1007C000898180FD02C085E0C2C02A8D3B8D4C8DA1
:1007D0005D8D8E899F89A88DB98D281B390B4A0B99
:1007E0005B0BCB01A0E0B0E0281739074A075B0795
:1007F00008F469015301412C72E0572EA0C02E89E4
:100800003F89488D598DDA01C9019170A070B0708F
:100810000097A105B10509F05EC0DA01C90169E0E0
:10082000B695A795979587956A95D1F7FA80FA942A
:10083000F822C9F4211531054105510529F46E8DC1
:100840007F8D88A199A105C06AA17BA18CA19DA1E2
:10085000FFDE623071058105910508F476C06AA358
:100860007BA38CA39DA300918200109183002AA1F9
:100870003BA14CA15DA12250304040405040F801C6
:1008800086819781A085B1850297A109B1092817B2
:1008900039074A075B0708F058C0628170E080E0C2
:1008A00090E0D4D49B01AC01F80182899389A4899A
:1008B000B589280F391F4A1F5B1F211531054105D6
:1008C000510509F442C02F0D311D411D511D2EA3AC
:1008D0003FA348A759A72E893F893170C201821BC7
:1008E000930B76018C159D0508F47C01611471044D
:1008F00019F480E090E001C0C5014EA15FA168A598
:1009000079A5870102DD882301F5C701A0E0B0E0E9
:100910002E893F89488D598D280F391F4A1F5B1F2B
:100920002E8B3F8B488F598FAE0CBF1CCE18DF0823
:10093000F401808191818E0D9F1D91838083C1146C
:10094000D10409F05CCF80E002C0198281E0DF9120
:10095000CF911F910F91FF90EF90DF90CF90BF90BC
:10096000AF909F908F907F906F905F904F90089581
:100970002F923F924F925F926F927F928F929F92AF
:10098000AF92BF92CF92DF92EF92FF920F931F939D
:10099000DF93CF93CDB7DEB7EF970FB6F894DEBFF6
:1009A0000FBECDBF4C0120908200309083002114F7
:1009B000310411F496E0B0C1F1011182CE0101962B
:1009C000988B8F8703C00894811C911CF40180814F
:1009D0008032C9F38F3219F40894811C911C198A52
:1009E0001A8A1B8A1C8AF4018081813248F4CE0164
:1009F0000D96B0DD982F1D8E882309F43AC18CC165
:100A0000CE0188969FAF8EAFAF85B889FD018BE090
:100A100090E002C020E2219301972FEF8F3F9207D1
:100A2000C9F738E01DAE20E002C03BE028E0F40149
:100A30008DADE80FF11D90818F5F8DAF9132B0F0D9
:100A40009F32A1F09E3211F0231728F0383071F454
:100A50009E3259F30BC0892F81568A3108F4905287
:100A6000FD01E20FF11D90832F5FE1CF1B961C92D9
:100A70001B97913218F491E01B969C93CE010D9632
:100A800069DD982F882309F0C9C0498D5A8D6B8D77
:100A90007C8D2D853E852F703070F5E0220F331F41
:100AA000FA95E1F7CE014D9600E210E02EDC8823A6
:100AB00009F056C18D8D882309F448C148A543FD2E
:100AC00012C02F853889D901FE017D968EAD9FAD6C
:100AD000E817F90709F43CC190818C91981719F433
:100AE00031961196F3CF0091820010918300AD846E
:100AF000BE840894A11CB11CA114B10409F426C140
:100B0000298D3A8D4B8D5C8D21153105410551059F
:100B100009F41CC1C5018F709070892B09F07BC04E
:100B20002F5F3F4F4F4F5F4F298F3A8F4B8F5C8F17
:100B30004D895E896F89788D411551056105710573
:100B400041F4F80184819581A816B90608F0FEC029
:100B500062C0F801828190E001979501E4E036954A
:100B60002795EA95E1F782239323892B09F053C057
:100B7000CB01BA016DDD9B01AC01623071058105CD
:100B8000910508F4EDC0F80186819781A085B185B3
:100B9000281739074A075B0708F0D8C02D8B3E8B12
:100BA0004F8B588FC0908200D09083006EEFE62E5E
:100BB0006FEFF62E6FEF062F6FEF162FE20EF31E7C
:100BC000041F151FF60186819781A085B1850297C4
:100BD000A109B109E816F9060A071B0728F020E069
:100BE00030E040E050E013C0F601228130E040E008
:100BF00050E0C801B7012AD39B01AC01F6018289FC
:100C00009389A489B589280F391F4A1F5B1F298F33
:100C10003A8F4B8F5C8FBE86AD8637CF833009F01D
:100C20007BC0EF85F8898385882309F497C074C059
:100C300044FF94C0FDAD8F0E911C5AA8442429A9ED
:100C400030E02429352940E050E0A901332722274C
:100C500078AC66248FA990E086299729A0E0B0E0BF
:100C6000282B392B4A2B5B2B298B3A8B4B8B5C8B9C
:100C7000CBCE8D8D882309F44EC088A584FD4BC052
:100C80003AA920E089A990E0282B392B40E050E0D8
:100C9000A9013327222798AD80E06FA970E0862B49
:100CA000972BA0E0B0E0282B392B4A2B5B2BF101CE
:100CB000268F378F40A351A32CAD30E040E050E0A9
:100CC000522F4427332722278BAD90E0A0E0B0E0DD
:100CD000DC0199278827282B392B4A2B5B2B89ADE0
:100CE00090E0A0E0B0E0282B392B4A2B5B2B9AAD8B
:100CF00080E0A0E0B0E0282B392B4A2B5B2B228F21
:100D0000338F448F558F168A178A108E118E81E08B
:100D1000818390E001C093E0892FEF960FB6F8949D
:100D2000DEBF0FBECDBFCF91DF911F910F91FF901E
:100D3000EF90DF90CF90BF90AF909F908F907F907B
:100D40006F905F904F903F902F90089593E069CF00
:100D5000F9018385882309F46BCF8BCF94E0DCCF36
:100D600091E0DACFCF92DF92EF92FF920F931F9331
:100D7000CF93DF93EC016A017B012EEF31E002E0BB
:100D800010E0C3DA882311F043E039C0998180E094
:100D9000288130E0822B932B85559A4A11F042E04E
:100DA0002EC0CE01B701A60126E330E002E010E03C
:100DB000ACDA882359F4998180E0288130E0822BD5
:100DC000932B8654914411F440E019C0CE01B70131
:100DD000A60122E530E002E010E097DA882311F066
:100DE00041E00DC040E0998180E0288130E0822B15
:100DF000932B8654914409F441E081E04827842FE5
:100E0000DF91CF911F910F91FF90EF90DF90CF90E6
:100E100008954F925F926F927F928F929F92AF92BE
:100E2000BF92CF92DF92EF92FF920F931F93DF93C7
:100E3000CF93CDB7DEB7A4970FB6F894DEBF0FBE41
:100E4000CDBF4C011092830010928200009709F4EC
:100E50007CC1BCDA80FF02C082E07CC17E010894C4
:100E6000E11CF11CC70140E050E060E070E07ADF77
:100E7000813021F0AA24BB24650138C0C70140E0BD
:100E800050E060E070E02EEB31E000E110E03DDA90
:100E9000882309F05CC18D81882309F45AC18C85AF
:100EA00090E0A0E0B0E0D82ECC24BB24AA248B850F
:100EB00090E0A0E0B0E0DC0199278827A82AB92AB1
:100EC000CA2ADB2A898590E0A0E0B0E0A82AB92AE6
:100ED000CA2ADB2A9A8580E0A0E0B0E0A82AB92AD5
:100EE000CA2ADB2AC701B601A5013CDF833009F419
:100EF0002EC1882309F02DC1CE010196B601A501AE
:100F00002DE030E004E210E000DA882309F01FC190
:100F10009B8580E02A8530E0822B932B7C0100E0CA
:100F200010E0E114F1040105110519F58B8D90E035
:100F3000A0E0B0E0182F0027FF24EE248A8D90E077
:100F4000A0E0B0E0DC0199278827E82AF92A0A2BDB
:100F50001B2B888D90E0A0E0B0E0E82AF92A0A2B4C
:100F60001B2B998D80E0A0E0B0E0E82AF92A0A2B3B
:100F70001B2B2C8130E040E050E0C801B70166D166
:100F80002B013C019B8180E02A8130E0822B932B56
:100F9000A0E0B0E0A80EB91ECA1EDB1EF401A286B6
:100FA000B386C486D586898182839E8180E02D8127
:100FB000422F50E0482B592B55834483988580E07D
:100FC0002F8130E0822B932B7C0100E010E0E114B4
:100FD000F1040105110519F58F8990E0A0E0B0E05A
:100FE000182F0027FF24EE248E8990E0A0E0B0E0C7
:100FF000DC0199278827E82AF92A0A2B1B2B8C89E0
:1010000090E0A0E0B0E0E82AF92A0A2B1B2B9D898A
:1010100080E0A0E0B0E0E82AF92A0A2B1B2B9B8194
:1010200080E02A8130E0822B932BA0E0B0E0E81A28
:10103000F90A0A0B1B0BE418F5080609170984E0E6
:10104000569547958A95E1F7CA01A0E0B0E0E81A05
:10105000F90A0A0B1B0BF401228130E040E050E05A
:10106000C801B70112D12E5F3F4F4F4F5F4FF401C0
:101070002683378340875187273FFFE03F07F0E013
:101080004F07F0E05F0708F464C0275F3F4F404020
:10109000504010F083E001C082E0F401808383308F
:1010A00041F52BA130E040E050E0522F4427332798
:1010B00022278AA190E0A0E0B0E0DC0199278827F0
:1010C000282B392B4A2B5B2B88A190E0A0E0B0E0C5
:1010D000282B392B4A2B5B2B99A180E0A0E0B0E0B4
:1010E000282B392B4A2B5B2B26873787408B518B3C
:1010F0000DC0F40182859385A485B585840D951D69
:10110000A61DB71D86879787A08BB18BF4018481BC
:101110009581A4E096958795AA95E1F7A0E0B0E0C7
:101120002285338544855585820F931FA41FB51FE3
:10113000840D951DA61DB71D828B938BA48BB58B3B
:101140001182909283008092820080E003C081E04F
:1011500001C087E0A4960FB6F894DEBF0FBECDBFE6
:10116000CF91DF911F910F91FF90EF90DF90CF9083
:10117000BF90AF909F908F907F906F905F904F90B7
:10118000089587B38C6287BBBC9888B38C6388BB97
:1011900080E58DB981E08EB908958FB9779BFECF38
:1011A00008958FEF8FB9779BFECF8FB108958FB9D8
:1011B000779BFECF8FB10895982FFB0106C08081E9
:1011C0008FB9779BFECF319691509923C1F708953F
:1011D000982FFB0107C080818FB9779BFECF8FB11D
:1011E000819391509923B9F7089584B3807F84BB8C
:1011F00085B38F6085BB0895989902C091E00BC0BC
:101200009A9902C093E007C0999902C092E003C086
:101210009B9911C094E080918500873420F08EE383
:101220008093850005C08F5F80938500843029F40A
:101230009093840008951092850008958091840011
:10124000109284000895809384000895629FD001D5
:10125000739FF001829FE00DF11D649FE00DF11D71
:10126000929FF00D839FF00D749FF00D659FF00D20
:101270009927729FB00DE11DF91F639FB00DE11D0D
:10128000F91FBD01CF0111240895A1E21A2EAA1B56
:10129000BB1BFD010DC0AA1FBB1FEE1FFF1FA21726
:1012A000B307E407F50720F0A21BB30BE40BF50B23
:1012B000661F771F881F991F1A9469F760957095AC
:1012C000809590959B01AC01BD01CF010895F894E4
:0212D000FFCF4E
:1012D200317A762E77617600327A762E77617600D1
:1012E200337A762E77617600347A762E77617600BD
:00000001FF
